:020000040000FA
:0400000080312528FE
:080008009110250082317C03F8
:100010000A0091008A0A7C030A009300880A8A0A6F
:100020007C030A0091008A0A7C030A0093008A0A72
:100030007C030A0098008A0A7C030A009A00FC0BE1
:100040000900B430FC00FD0A090023008C018D0179
:1000500020008C018D0191013F309B00B430FC00E9
:10006000250082317C030A0091008A0A7C030A0081
:100070009300203098000C309A00880A8A0A7C038A
:100080000A0091008A0A7C030A0093008A0A7C0312
:100090000A0098008A0A7C030A009A008031200036
:1000A000FC0321000830950091148C018D01200083
:1000B0003C309A002000FD010B178B171C15FD1F0B
:0600C0005F280C14622809
:100400002034213422342334243425342634273430
:100410002834293429342A342B342C342D342E34E6
:100420002F3430343134313432343334343434349E
:100430003534363436343734373438343934393463
:1004400039343A343A343B343B343B343C343C3436
:100450003C343C343C343C343C343C343C343C341C
:100460003C343C343C343C343C343B343B343B340F
:100470003A343A3439343934393438343734373417
:10048000363436343534343434343334323431342D
:10049000313430342F342E342D342C342B342A3450
:1004A0002934293428342734263425342434233479
:1004B0002234213420341F341E341D341C341B34A8
:1004C0001A341934183417341634153414341334D8
:1004D00012341134103410340F340E340D340C3403
:1004E0000C340B340A340A34093408340834073421
:1004F0000734063406340534053405340434043432
:100500000434043403340334033403340334033431
:100510000334033403340334033404340434043420
:1005200004340534053405340634063407340734FE
:100530000834083409340A340A340B340C340C34CB
:100540000D340E340F34103410341134123413348B
:100550001434153416341734183419341A341B343F
:0C0560001C341D341E341F3420342134A0
:100600000C340C340C340C340C340C340C340C34EA
:100610000C340C343C343C343C342C342C341C34FA
:100620001C340C340C343C342C341C340C343C342A
:100630001C340C343C341C343C342C340C342C34FA
:100640003C341C343C340C341C343C340C340C34FA
:100650001C342C342C343C343C343C343C343C345A
:100660002C342C341C340C340C343C341C340C34FA
:100670003C341C343C342C340C342C343C341C348A
:100680003C340C341C343C340C341C342C343C349A
:100690000C340C341C341C342C342C343C343C349A
:1006A0003C340C340C340C340C340C340C340C341A
:1006B0000C340C340C340C340C340C340C340C343A
:1006C0000C340C340C340C341C341C341C342C34DA
:1006D0002C343C343C340C340C341C342C343C343A
:1006E0000C341C343C340C341C343C341C342C345A
:1006F0000C342C341C343C341C340C343C341C344A
:100700000C340C343C342C342C341C341C341C3449
:100710001C341C342C342C343C340C340C341C3439
:100720003C340C341C343C341C342C340C342C3409
:100730001C343C341C340C343C341C340C343C34F9
:100740002C341C340C340C343C342C342C342C34E9
:100750001C341C341C340C340C340C340C340C3469
:0C0760000C340C340C340C340C340C340D
:100800003934383437343734363436343534343494
:100810003434333432343134313430342F342E34B0
:100820002D342C342B342A342934293428342734D9
:1008300026342534243423342234213420341F3404
:100840001E341D341C341B341A3419341834173434
:100850001634153414341334123411341034103463
:100860000F340E340D340C340C340B340A340A3487
:1008700009340834083407340734063406340534A0
:1008800005340534043404340434043403340334A8
:1008900003340334033403340334033403340334A0
:1008A0000334043404340434043405340534053486
:1008B00006340634073407340834083409340A345B
:1008C0000A340B340C340C340D340E340F34103421
:1008D00010341134123413341434153416341734DC
:1008E000183419341A341B341C341D341E341F348C
:1008F000203421342234233424342534263427343C
:100900002834293429342A342B342C342D342E34F1
:100910002F343034313431343234333434343434A9
:10092000353436343634373437343834393439346E
:1009300039343A343A343B343B343B343C343C3441
:100940003C343C343C343C343C343C343C343C3427
:100950003C343C343C343C343C343B343B343B341A
:0C0960003A343A343934393439343834FC
:100A00000C342C343C341C343C340C341C343C3416
:100A10000C341C342C343C340C340C341C342C3446
:100A20002C342C343C343C343C340C340C340C34F6
:100A30000C340C340C340C340C340C340C340C34B6
:100A40000C340C340C340C340C340C340C340C34A6
:100A50001C341C341C342C342C343C343C340C34C6
:100A60000C341C342C343C340C341C343C340C34E6
:100A70001C343C341C342C340C342C341C343C34A6
:100A80001C340C343C341C340C340C343C342C34C6
:100A90002C341C341C341C341C341C342C342C34A6
:100AA0003C340C340C341C343C340C341C343C3496
:100AB0001C342C340C342C341C343C341C340C3496
:100AC0003C341C340C343C342C341C340C340C3486
:100AD0003C342C342C342C341C341C341C340C3456
:100AE0000C340C340C340C340C340C340C340C3406
:100AF0000C340C340C340C340C340C340C340C34F6
:100B00000C340C343C343C343C342C342C341C3405
:100B10001C340C340C343C342C341C340C343C3435
:100B20001C340C343C341C343C342C340C342C3405
:100B30003C341C343C340C341C343C340C340C3405
:100B40001C342C342C343C343C343C343C343C3465
:100B50002C342C341C340C340C343C341C340C3405
:0C0B60003C341C343C342C340C342C3459
:100C0000073406340634053405340534043404341A
:100C1000043404340334033403340334033403341A
:100C20000334033403340334033404340434043409
:100C300004340534053405340634063407340734E7
:100C40000834083409340A340A340B340C340C34B4
:100C50000D340E340F341034103411341234133474
:100C60001434153416341734183419341A341B3428
:100C70001C341D341E341F342034213422342334D8
:100C800024342534263427342834293429342A348A
:100C90002B342C342D342E342F3430343134313441
:100CA00032343334343434343534363436343734FF
:100CB000373438343934393439343A343A343B34CB
:100CC0003B343B343C343C343C343C343C343C34A6
:100CD0003C343C343C343C343C343C343C343C3494
:100CE0003C343B343B343B343A343A343934393491
:100CF00039343834373437343634363435343434A0
:100D00003434333432343134313430342F342E34BB
:100D10002D342C342B342A342934293428342734E4
:100D200026342534243423342234213420341F340F
:100D30001E341D341C341B341A341934183417343F
:100D4000163415341434133412341134103410346E
:100D50000F340E340D340C340C340B340A340A3492
:0C0D600009340834083407340734063422
:100E00000C342C341C343C341C340C343C341C3432
:100E10000C340C343C342C342C341C341C341C3432
:100E20001C341C342C342C343C340C340C341C3422
:100E30003C340C341C343C341C342C340C342C34F2
:100E40001C343C341C340C343C341C340C343C34E2
:100E50002C341C340C340C343C342C342C342C34D2
:100E60001C341C341C340C340C340C340C340C3452
:100E70000C340C340C340C340C340C340C340C3472
:100E80000C340C340C340C340C340C343C343C3402
:100E90003C342C342C341C341C340C340C343C3492
:100EA0002C341C340C343C341C340C343C341C3492
:100EB0003C342C340C342C343C341C343C340C3452
:100EC0001C343C340C340C341C342C342C343C3462
:100ED0003C343C343C343C342C342C341C340C3402
:100EE0000C343C341C340C343C341C343C342C3432
:100EF0000C342C343C341C343C340C341C343C3422
:100F00000C341C342C343C340C340C341C341C3461
:100F10002C342C343C343C343C340C340C340C3401
:100F20000C340C340C340C340C340C340C340C34C1
:100F30000C340C340C340C340C340C340C340C34B1
:100F40001C341C341C342C342C343C343C340C34D1
:100F50000C341C342C343C340C341C343C340C34F1
:0E0F60001C343C341C342C340C342C34B62F8E
:020000040001F9
:02000E0082C9A5
:02001000FFDC13
:00000001FF
